:020000040000FA
:06000000F8EF06F012000B
:06080000F8EF06F0120003
:06082A000100240E000095
:0808300000020000200000009E
:08083800D9CFE6FFE1CFD9FFA3
:10084000040EE126DE6ADE6ADE6ADD6ADD52DD5212
:10085000FD0EDBCF00F0FE0EDBCF01F0026A036A73
:1008600001AE02D002680368D9CFE9FFDACFEAFF10
:10087000030EEB500318E8AE02D0033408D000504A
:10088000EE5C0150EE580250EE580350EE580FE265
:100890000C0EE66ED8EC06F0E552D9CFE9FFDACFC0
:1008A000EAFFEE2A000EEE22EE22EE22D1D7040E4F
:1008B000E15C02E2E16AE552E16EE552E7CFD9FF81
:1008C00012000F0EC16E070EB46E936A300E926E58
:1008D0000F0E946EF19E816A80901200D9CFE6FFD0
:1008E000E1CFD9FF020EE1268250020B01E0010E9A
:1008F000080DF3CF02F08250010B040DF3CF01F08D
:100900008050200B01E0010EE824006E8050100B97
:1009100001E0010E002401240224DE6EDD6ADECF38
:1009200000F0DDCF01F000C0F3FF01C0F4FF020EC4
:10093000E15C03E200D0E16AE552E16EE552E7CF07
:10094000D9FF12008092320EE66E06EC07F0E552F7
:100950008084320EE66E06EC07F0E5528094320E8B
:10096000E66E06EC07F0E55212008082320EE66E6B
:1009700006EC07F0E5528084320EE66E06EC07F0D6
:10098000E5528094320EE66E06EC07F0E552120056
:10099000380E816ED7DF320EE66EE66A4DDFE55225
:1009A000E552010E816ECEDF320EE66EE66A44DF5E
:1009B000E552E5520D0E816EC5DF320EE66EE66A37
:1009C0003BDFE552E552060E816EBCDF320EE66E6D
:1009D000E66A32DFE552E5521200010E816EB2DFA7
:1009E0000A0EE66EE66A28DFE552E5521200D9CF1C
:1009F000E6FFE1CFD9FF020E816EA4DF0A0EE66E9C
:100A0000E66A1ADFE552E552FD0EDBCFE6FFFE0E89
:100A1000DB50280DF350E552E724E76EFE0EE7CFDA
:100A2000DBFFFD0EDB6AFE0EDB50F36EFD0EDBCF4F
:100A3000F4FFF350F45C0BE2140E816E83DF320E90
:100A4000E66E06EC07F0E552FD0EDB2AECD7E55228
:100A5000E7CFD9FF1200D9CFE6FFE1CFD9FFFE0ED5
:100A6000DB50816E82DF320EE66E06EC07F0E55257
:100A7000E552E7CFD9FF1200D9CFE6FFE1CFD9FF8A
:100A8000FD0EDBCFE9FFFE0EDBCFEAFFEF500EE0FD
:100A9000FD0EDBCFE9FFDB2AFE0EDBCFEAFF01E331
:100AA000DB2AEF50E66ED7DFE552EAD7E552E7CF13
:100AB000D9FF12000201246B300E926EF00E936E7D
:100AC000EF0E206F20C281FF040E216F215100081C
:100AD00021E22051FE0BE842206F20C281FF050E6B
:100AE000E66EE66AA9DEE552E5528150100B09E098
:100AF0008150200B06E08150400B03E08150800BB9
:100B000001E10AD80201240502E1255104D02105A2
:100B1000216FDCD7CFD71200F00E936E81CF23F276
:100B200002012315226F0F0E2015206F2051221174
:100B3000206F81CF23F2F00E2315226FF00E225D7D
:100B400001E0F7D7936A06D826C225F20201010E0A
:100B5000246F12000201276B100E275D14E227514B
:100B6000EA6A000FE96E020EEA22EF50205D08E10A
:100B70002751EA6A100FE96E020EEA22EFCF26F241
:100B80002729276FE9D726C281FF640EE66EE66A41
:100B900053DEE552E55212000201286B070E285D74
:100BA0001DE288DF0201296F2851EA6A2A0FE96EE7
:100BB000020EEA2229C2EFFF2851EA6A2A0FE96EE3
:100BC000020EEA22EF50460802E108D004D029C202
:100BD000E6FF41DFE5520201282BE0D72851EA6AFF
:100BE0002A0FE96E020EEA22EF6A12000201286B58
:100BF000070E285D16E22851EA6A2A0FE96E020EF6
:100C0000EA22EF50E66E27DFE55202012829EA6A60
:100C10002A0FE96E020EEA22EF5001E102D0282BE2
:100C2000E7D71200D9CFE6FFE1CFD9FFE652F25065
:100C3000800B01E0010EDF6EF29EA69EA69CA684AC
:100C4000FE0EDB50A96EFD0EDB50A86E550EA76E92
:100C5000AA0EA76EA682A6B2FED7A694DF50E8B071
:100C6000F28EE8A0F29EE552E552E7CFD9FF1200DE
:100C7000D9CFE6FFE1CFD9FFA69CA69EFE0EDB50A2
:100C8000A96EA680A85000D0E552E7CFD9FF120088
:100C900018DE818080B81ED081AE08D08180819E10
:100CA000FA0EE66EE66AC8DDE552E5528150E824A8
:100CB000816EFA0EE66EE66ABFDDE552E55281AE60
:100CC00008D08180819EFA0EE66EE66AB5DDE552B7
:100CD000E5521DD081A008D08190818EFA0EE66E7B
:100CE000E66AAADDE552E55281407F0B816EFA0E7D
:100CF000E66EE66AA1DDE552E55281A008D0818E5C
:100D00008190FA0EE66EE66A97DDE552E552C2D7AB
:020D10001200CF
:0E0D12002A0EF66E080EF76E000EF86E020145
:100D20000900F550386F0900F550396F03E1386755
:100D300001D03DD00900F550336F0900F550346FF4
:100D40000900F550356F09000900F550E96E0900FA
:100D5000F550EA6E090009000900F550366F0900E8
:100D6000F550376F09000900F6CF3AF2F7CF3BF2A2
:100D7000F8CF3CF233C2F6FF34C2F7FF35C2F8FFBA
:100D80000201365302E1375307E00900F550EE6ED9
:100D90003607F8E23707F9D73AC2F6FF3BC2F7FF4A
:100DA0003CC2F8FF02013807000E395BBFD71200C2
:100DB000FF0EE350066E480E01D04C0EE76EE72E94
:100DC000FED7E76AE72EFED7062EF7D700001200FF
:100DD000000EF36E00EE00F0080E01D81200EA607B
:100DE00002D0EE6AFCD7F350E9601200EE6AFCD73D
:100DF00012EE40F022EE40F0F86A059C89EC06F015
:0C0E000011EC07F048EC06F0FBD71200E4
:040E0C00FF0EE350A2
:100E1000E84E1200000000D000D000D0E82EFAD733
:020E20001200BE
:020E22001200BC
:0C0E2400EEEDEBE7DEDDDBD7BEBDBBB7BB
:100E30007E7D7B7730313233343536373839414235
:040E4000434445469C
:00000001FF
